:020000040000FA
:020000000528D1
:06000A008312850183163C
:10001000CB30850071308F0053309F00FF3092004D
:10002000831283120730990001309F0093010C3036
:10003000950004309200A601FF30A2009F111F110D
:100040009F149F1821281F151E08A6008030A602A5
:1000500003182D28A6090130A607000000000000A3
:100060000000000000000000000000000000000090
:10007000000000009F149F183B281F111E08A500B8
:100080002508A3005C20A1006821A0000310A60D94
:10009000031C4C28FF30A600260893002208A60265
:1000A00003185728051285162108A20020280516D6
:1000B00085122008A20020282308A4006830A40785
:1000C00000300318013E8A002408672008008200DF
:1000D0001D341E341F341F34203421342234233481
:1000E00024342534263426342734283429342A3439
:1000F0002B342C342D342D342E342F3430343134F1
:1001000032343334343434343534363437343834A8
:1001100039343A343B343C343C343D343E343F345F
:100120004034413442344334433444344534463417
:100130004734483449344A344A344B344C344D34CF
:100140004E344F3450345134513452345334543487
:100150005534563457345834583459345A345B343F
:100160005C345D345E345F345F34603461346234F7
:1001700063346434653466346734673468346934AE
:100180006A346B346C346D346E346E346F34703466
:10019000713472347334743475347534763477341E
:1001A000783479347A347B347C347C347D347E34D6
:1001B0007F3480348134823483348334843485348E
:1001C00086348734883489348A348A348B348C3446
:1001D0008D348E348F3490349134923492349334FD
:1001E00094349534963497349834993499349A34B5
:1001F0009B349C349D349E349F34A034A034A1346D
:10020000A234A334A434A534A634A734A734A83424
:10021000A934AA34AB34AC34AD34AE34AE34AF34DC
:10022000B034B134B234B334B434B534B534B63494
:10023000B734B834B934BA34BB34BC34BD34BD344B
:10024000BE34BF34C034C134C234C334C434C43403
:10025000C534C634C734C834C934CA34CB34CB34BB
:10026000CC34CD34CE34CF34D034D134D234D23473
:10027000D334D434D534D634D734D834D934D9342B
:10028000DA34DB34DC34DD34DE34DF34E034E034E3
:10029000E134E234E334E434E534E634E734E8349A
:1002A000E834E934EA34EB34EC34ED34EE34EF3452
:1002B000EF34F034F134F234F334F434F534F6340A
:1002C000F634F734F834F934FA34FB34FC34FD34C2
:1002D0002308A4007430A40701300318013E8A00EB
:1002E0002408732108008200163417341834183497
:1002F00019341A341A341B341C341D341D341E3482
:100300001F341F3420342134213422342334233445
:10031000243425342534263427342734283429340A
:100320002A342A342B342C342C342D342E342E34CD
:100330002F34303430343134323432343334343492
:100340003434353436343634373438343934393457
:100350003A343B343B343C343D343D343E343F341A
:100360003F344034413441344234433443344434E0
:1003700045344534463447344834483449344A34A3
:100380004A344B344C344C344D344E344E344F3468
:10039000503450345134523452345334543455342C
:1003A00055345634573457345834593459345A34F0
:1003B0005B345B345C345D345D345E345F345F34B5
:1003C0006034613461346234633464346434653479
:1003D0006634663467346834683469346A346A343D
:1003E0006B346C346C346D346E346E346F34703402
:1003F00070347134723473347334743475347534C6
:100400007634773477347834793479347A347B3489
:100410007B347C347D347D347E347F34803480344E
:100420008134823482348334843484348534863411
:10043000863487348834883489348A348A348B34D7
:100440008C348C348D348E348F348F34903491349A
:10045000913492349334933494349534953496345F
:10046000973497349834993499349A349B349B3424
:100470009C349D349E349E349F34A034A034A134E7
:10048000A234A234A334A434A434A534A634A634AC
:10049000A734A834A834A934AA34AB34AB34AC3470
:1004A000AD34AD34AE34AF34AF34B034B134B13434
:1004B000B234B334B334B434B534B534B634B734F9
:1004C000B734B834B934BA34BA34BB34BC34BC34BD
:1004D000BD34BE34BE34BF34C034C034C134C23481
:0804E000C234C334C434C43437
:02400E00C430BC
:00000001FF
